:020000040000FA
:10000000850186018316073085008601831207303B
:100010009F001D2882076F340334763457341B3415
:100020005D347D3407347F345F343F3479346C344D
:1000300073347C343C3468343E34A301A501A401FC
:100040005B20051C302805192128051C3028051DBA
:100050002528A30A103023020318A3015B202128BE
:10006000A4175B20851832281030A50060200C30C2
:100070002307A2004520A20B3A28A4011130A500B5
:1000800060208517502085131D28FA30A000C83045
:10009000A10000000000A10B4928A00B4728080080
:1000A000FA30A000C830A10000000000A10B5428C5
:1000B000A00B5228080023080A2024048600080008
:0A00C00025080A2024048600080029
:02400E00703F01
:00000001FF
